:100000000C9475070C9492070C9492070C94722C24
:100010000C9492070C9492070C9492070C949207FC
:100020000C9492070C9492070C9445220C9487210F
:100030000C9489250C9492070C9492070C949207C7
:100040000C9492070C9492070C9492070C949207CC
:100050000C9492070C943C250C9492070C949207F4
:100060000C9492070C9492070C9492070C949207AC
:100070000C9492070C9492070C9492070C9492079C
:100080000C9492070C9492070C9492070C9492078C
:100090000C9492070C9492070C9492070C9492077C
:1000A0000C9492070C9492070C949207E10A550B5A
:1000B000E90AB30AB70AED0ABA0AF00AFB0AC50A46
:1000C0004B0BC90AFF0ACD0A030B2D0BD10A070BF4
:1000D000370BD70A0D0B170BBE0AF40AC10AF70A31
:1000E000DC0A120B230B430B450BAF0AE50A5E0B30
:1000F000840B8A0B780B7E0B900B960B9C0B540C8D
:10010000540C870C870C010D1F0D270E270E240D94
:10011000980DA90DA90D0C120F12381248124F128A
:100120005A12F012F012F012F012F0125D125F1279
:1001300064128812A912AC12AF12D112991FC01FFB
:100140006F21C01F6F210C202F206F212521352109
:1001500090297E29A229FE285B2A5B2A7B295B2A1B
:100160005B2ACF295B2AE329392A5B2A5B2A5B2A8F
:100170005B2A0D2A5B2A5B2AFE295B2ABB295B2AA4
:100180005B2A552A552A552A552A552A552A552A71
:10019000552A552A572A5B2A902973295B2A5B2AFC
:1001A0005B2A5B2A5B2A5B2A5B2A5B2A5B2A5B2A27
:1001B000572A5B2A5B2A7B295B2A532A532A532A14
:1001C000532A532A532A532A532A532A572A0000C0
:1001D000000000000000000000000000000000001F
:1001E000000000000000000000000000000000000F
:1001F00000007E0F00D4FFFFFFC700000078000062
:100200000000000000002A2B280000000000000071
:1002100000000000000000000029000000002C1E6B
:100220003420212224342627252E362D3738271E28
:100230001F202122232425263333362E37381F044E
:1002400005060708090A0B0C0D0E0F1011121314E6
:1002500015161718191A1B1C1D2F3130232D3504A4
:1002600005060708090A0B0C0D0E0F1011121314C6
:1002700015161718191A1B1C1D2F3130354C444503
:100280004255473A2064697361626C65642E0A00C6
:1002900044454255473A20656E61626C65642E0A9A
:1002A000005B735D000A002530313662003A2000A1
:1002B00025303258000A722F632030313233343502
:1002C000363738394142434445460A000A00253052
:1002D0003258006C65645F7461736B3A20004F6E36
:1002E0006573686F743A206163746976653A202596
:1002F000640A000A002530325820006B6579626F6D
:100300006172645F7265706F72743A20005461723A
:1003100067657420636F6E6E65637465640D0A00B3
:1003200054617267657420646973636F6E6E656390
:100330007465642C207468726F74746C696E6720C5
:10034000636F6E6E656374696F6E20617474656D42
:100350007074730D0A004661696C656420746F20C7
:10036000657865637574652025730A003F00433E18
:1003700020000631FF0974A1010975150026FF0050
:100380009520750881020976150026FF00952075D5
:10039000089102C005010902A10185020901A1001D
:1003A0000509190129081500250195087501810223
:1003B0000501093009311581257F950275088106EF
:1003C00009381581257F950175088106050C0A38C5
:1003D000021581257F950175088106C0C0050109B8
:1003E00080A101850319012AB700150126B70095E0
:1003F0000175108100C0050C0901A10185041901D6
:100400002AA002150126A002950175108100C005E1
:10041000010906A1018506050719E029E715002550
:10042000019508750181020507190029EF150025BE
:100430000195F075018102050819012905950575D9
:10044000019102950175039101C00660FF0961A148
:10045000010962150026FF009520750881020963D5
:10046000150026FF00952075089102C005010906B8
:10047000A101050719E029E7150025019508750177
:1004800081029501750881010507190029FF1500F2
:1004900026FF0095067508810005081901290595B4
:1004A0000575019102950175039101C05B435D00E3
:1004B0005B445D005B535D005B575D005B525D001C
:1004C00009027B00040100A0FA09040000010301F5
:1004D00001000921110100012240000705810308E4
:1004E00000010904010002030000000921110100BC
:1004F00001222200070582032000010705030320D3
:10050000000109040200010300000009211101009B
:100510000122B6000705840320000109040300023C
:1005200003000000092111010001222200070585B6
:10053000032000010705050320000112010002004D
:100540000000086C6101000100010200010E03427D
:10055000007200650065007A00650000001C034120
:100560000066007400650072006E006F006F006E20
:10057000004C006100620073000000040309047075
:100580003A097072696E742076616C7565730A64DD
:100590003A097365742064656661756C74730A75D5
:1005A000703A092B310A646E3A092D310A6C743A9B
:1005B000092B31300A72743A092D31300A45534300
:1005C0002F713A09717569740A0A73706565642040
:1005D0003D2064656C7461202A206D61785F7370C2
:1005E000656564202A2028726570656174202F205B
:1005F00074696D655F746F5F6D6178290A776865EE
:1006000072652064656C74613A20637572736F72F1
:100610003D25642C20776865656C3D25640A53652B
:100620006520687474703A2F2F656E2E77696B6938
:1006300070656469612E6F72672F77696B692F4DE2
:100640006F7573655F6B6579730A004D3E20004DD1
:1006500025753A25733E20003F0A003D2025750A86
:10066000003F0A0064656661756C74730A00257545
:100670000A003F0A000A092D2056616C7565732037
:100680002D0A00710A000A092D204D6F7573656BE4
:100690006579202D0A004C25640A002200210020E3
:1006A000001F001E002900000000000000170015B8
:1006B0000008001A0014002B000000000000000ACF
:1006C000000900070016000400E000000000000020
:1006D000000500190006001B001D00E100000000DD
:1006E0000000002C00E300E200E000000000000039
:1006F0000000000000230024002500260027002A17
:10070000002D002E0035001C0018000C00120013F4
:10071000004C002F00300031000B000D000E000FC8
:1007200000330034000000520000001100100036B9
:100730000037003800E500500051004F002800222B
:1007400052215200000000000000000000000001E3
:10075000000100010001000100007C000000000019
:100760000001000100010001000100010000000083
:100770000000000100010001000100010001000073
:100780000000000000010001000100010001000163
:100790000000000000000001000100010001000055
:1007A0000000000000000000000100010001000145
:1007B0000001000100A800AA00A900010001000139
:1007C0000001000100010001000100010001000121
:1007D0000001000100010001000000010000000113
:1007E0000001000100010001000100010001000101
:1007F00000010001000100010000000000000000F5
:1008000000000001000100010001000100010000E2
:1008100000000000000100010001000100010001D2
:1008200000000000000000010001000100010001C3
:1008300000010000000000000001000100010001B3
:1008400000010001000000000000000100010001A3
:10085000000100000000000000000000000100672F
:100860000054005500560001000100010001000184
:10087000005F0060006100570001000100010001FD
:100880000001005C005D005E00010001000000014D
:10089000000000010059005A005B00010001000146
:1008A000000100010001000100620063000000007F
:1008B0000000000000000001000100010001000133
:1008C0000001000000000000000100010001000123
:1008D0000001000100000000000000010001000113
:1008E0000001000100010000000000000001000103
:1008F00000010001000100010000000000000001F3
:1009000000010001000100000000000000000000E4
:1009100000010001000100010001000100010001CF
:1009200000010001000100010001000100010001BF
:1009300000010001000100010001000100010001AF
:1009400000000001000000010001000100010001A1
:10095000000100010001000100010001000100018F
:1009600000000000000000000000006164645F6B94
:1009700065795F6269743A2063616E2774206164EF
:10098000643A20253032580A0064656C5F6B6579E3
:100990005F6269743A2063616E27742064656C3A03
:1009A00020253032580A00290A002575002F00251D
:1009B00075005D28002564002000256400200025C6
:1009C000640020002564007C0025303258006D6FE3
:1009D0007573656B6579205B62746E7C7820792015
:1009E0007620685D287265702F61636C293A205B00
:1009F000006B65796D61705F636F6E6669672E72FB
:100A000061773A20253032580A2E737761705F6320
:100A10006F6E74726F6C5F636170736C6F636B3A4F
:100A20002025750A2E636170736C6F636B5F746F42
:100A30005F636F6E74726F6C3A2025750A2E737740
:100A400061705F6C63746C5F6C6775693A202575C3
:100A50000A2E737761705F7263746C5F7267756979
:100A60003A2025750A2E737761705F6C616C745F34
:100A70006C6775693A2025750A2E737761705F720D
:100A8000616C745F726775693A2025750A2E6E6F06
:100A90005F6775693A2025750A2E737761705F6705
:100AA000726176655F6573633A2025750A2E7377E8
:100AB00061705F6261636B736C6173685F626163D5
:100AC0006B73706163653A2025750A2E6E6B726FC9
:100AD0003A2025750A2E737761705F6573636170C4
:100AE000655F636170736C6F636B3A2025750A00F4
:100AF00064656275675F636F6E6669672E726177A2
:100B00003A20253032580A2E656E61626C653A20B3
:100B100025750A2E6D61747269783A2025750A2E42
:100B20006B6579626F6172643A2025750A2E6D6F6C
:100B30007573653A2025750A006565636F6E666991
:100B4000673A0A64656661756C745F6C6179657299
:100B50003A2025750A000A092D204D616769632036
:100B60002D0A443A094465627567204D65737361C7
:100B7000676520546F67676C650A583A094D617460
:100B8000726978204465627567204D6F64652054F2
:100B90006F67676C65202D2053686F77206B6579D0
:100BA0007072657373657320696E206D617472690C
:100BB0007820677269640A4B3A094B6579626F6104
:100BC000726420446562756720546F67676C6520A6
:100BD0002D2053686F77206B657970726573732071
:100BE0007265706F72740A4D3A09446562756720C8
:100BF0004D6F75736520546F67676C650A563A09C7
:100C000056657273696F6E0A533A0953746174754D
:100C1000730A433A09416374697661746520436FCE
:100C20006E736F6C65204D6F64650A46312D4631D9
:100C3000303A0953776974636820746F204C617986
:100C4000657220302D392028463130203D204C302F
:100C5000290A302D393A0953776974636820746F13
:100C6000204C6179657220302D390A475241564532
:100C70003A0953776974636820746F204C61796511
:100C80007220302028616C7465726E617465290A67
:100C9000423A094A756D7020746F20426F6F746C10
:100CA0006F616465720A4553433A094A756D702055
:100CB000746F20426F6F746C6F616465722028617D
:100CC0006C7465726E617465290A453A09507269DF
:100CD0006E7420454550524F4D2053657474696EB3
:100CE00067730A4241434B53504143453A09436CB1
:100CF00065617220454550524F4D0A4E3A094E4BA0
:100D0000524F20546F67676C650A000A092D204313
:100D10006F6E736F6C65202D0A4553432F713A092E
:100D2000717569740A6D3A096D6F7573656B6579D4
:100D30000A002573000A092D20537461747573200D
:100D40002D0A686F73745F6B6579626F6172645F9F
:100D50006C65647328293A20253032580A6B65790E
:100D6000626F6172645F70726F746F636F6C3A2050
:100D7000253032580A6B6579626F6172645F69640D
:100D80006C653A20253032580A6B65796D61705F69
:100D9000636F6E6669672E6E6B726F3A2025303214
:100DA000580A74696D65725F72656164333228290F
:100DB0003A202530386C580A003F004E4B524F3ACB
:100DC000206F66660A004E4B524F3A206F6E0A0043
:100DD0000A6D6F7573653A206F66660A000A6D6F5B
:100DE0007573653A206F6E0A000A6B6579626F61F0
:100DF00072643A206F66660A000A6B6579626F61F9
:100E000072643A206F6E0A000A6D61747269783AF2
:100E1000206F66660A000A6D61747269783A206F05
:100E20006E0A000A64656275673A206F66660A009A
:100E30000A64656275673A206F6E0A000A0A4A758D
:100E40006D70696E6720746F20626F6F746C6F6174
:100E50006465722E2E2E2000433E2000436C656197
:100E600072696E6720454550524F4D0A00313A096C
:100E700064656C6179282A31306D73293A202575B3
:100E80000A323A09696E74657276616C286D73294D
:100E90003A2025750A333A096D61785F737065658C
:100EA000643A2025750A343A0974696D655F746F78
:100EB0005F6D61783A2025750A353A09776865656E
:100EC0006C5F6D61785F73706565643A2025750AA3
:100ED000363A09776865656C5F74696D655F746F34
:100EE0005F6D61783A2025750A0011241FBECFEF8F
:100EF000DAE0DEBFCDBF12E0A0E0B1E0EAECFCE555
:100F000002C005900D92A23CB107D9F724E0A2ECF3
:100F1000B2E001C01D92AF32B207E1F70E947B0E32
:100F20000C94632E0C940000FF93EF93E091C202A7
:100F3000F091C302309709F00995EF91FF91089560
:100F4000FC018591803011F0EFDFFBCF0895FF2782
:100F5000E0E230E247FF0CC0419597FF09C0EDE2A7
:100F60006095709580959095611D711D811D911DF5
:100F700027FF02C0219530E350E2AA27660F771FB2
:100F8000881F991FAA1FA41710F0A41B63955A95D8
:100F9000A9F7AA3008F0A95FA05DAF93F39561159A
:100FA00071058105910541F7ED3211F4EF93F39549
:100FB000F21718F43F93F395FBCF8F91B5DFFA95B5
:100FC000E1F70895E991F9918591803021F085321A
:100FD00019F0AADFF9CF089520E0E8945591553231
:100FE000C1F3503311F4689455915A3348F4505377
:100FF00090F3220F022E220F220F200D250FF4CF87
:101000000EF4219589919991533619F3533729F1AB
:10101000533559F1BC0188279927E8945C3621F4AF
:101020008991999168945591543639F446EF7EF040
:1010300077FF0DC08FEF9FEF0AC055374AE039F0B8
:10104000583540E121F0523642E009F00895FF930F
:10105000EF937DDFEF91FF91B7CFFF93EF93FC010B
:1010600081918030B9F360DFFBCFFF93EF9368DFAE
:10107000F1CFDF93CF93CDB7DEB72596A3DFCF9126
:10108000DF9108950E94681C2FEF84E39CE02150BB
:1010900080409040E1F700C000009AE088E10FB680
:1010A000F894A895809360000FBE90936000FFCFE6
:1010B000A7E1B0E0EEE5F8E00C94A22D4B8B5C8B41
:1010C0006D8B7E8B8F8B611110924A0386E09E019F
:1010D000235F3F4FD901E82F1D92EA95E9F795E08C
:1010E000FE017396D90101900D929A95E1F79C89C2
:1010F0004E895F897B897D879E876F87598B488B57
:10110000F901DE01179601900D928A95E1F7CE0163
:1011100007960E943C1A81113EC086E0FE01379678
:10112000DE01119601900D928A95E1F7FF81E88525
:101130006A857B856115710531F0EF3F31F481E0FF
:10114000FF3F19F403C081E001C080E080FD23C0AF
:101150002091A50330E0C90101968770992740913D
:10116000D60350E08417950779F1F983EA837D83EC
:101170006C8396E0929FD001939FB00D1124AA55E5
:10118000BC4FFE01319601900D929A95E1F7809344
:10119000A5030E94561916E08091D6039091A503ED
:1011A0008917F9F0189FC00111248A559C4F0E949D
:1011B0003C1A8823B1F08091D60390E001968770A5
:1011C00099278093D603E8CF0E94681C1092A5034C
:1011D0001092D603EFE9F3E086E0DF011D928A95D5
:1011E000E9F76796E3E00C94BE2DADE0B0E0EBEFDD
:1011F000F8E00C94932DFC0180819181238134814E
:10120000232B31F09F3F31F491E08F3F19F403C05D
:1012100091E001C090E090FD58C57F0185E0DE01BE
:10122000199601900D928A95E1F7F701228189853F
:101230009A85222349F00E94C919182F682F8985A1
:101240009A850E94F71B03C00E94C31B182F698553
:101250007A85812F0E9481168C01F7018281882373
:1012600009F42CC19801225037472031310508F08C
:1012700041C18FEF93E00E94CA2D811129C1025014
:1012800036EFA32E32E0B32E002379F0A114F4E060
:10129000BF0609F41DC1C5010E94CA2D811101C0FC
:1012A00001502FEFA21AB20AEFCFCE0101962C0106
:1012B00088E0F20111928A95E9F72AE0322E850141
:1012C0000F5F1F4FC5010E94CA2D89831A82882390
:1012D00009F4FEC0813009F041C06501F2E0CF0E93
:1012E000D11CC8010E94CA2D8A83882309F4F0C04A
:1012F0009FEF980F933060F423E0A20EB11CC6015B
:101300000E94CA2D8B83882309F4E2C01C8229C065
:10131000843031F54E0133E0830E911C02E010E081
:1013200056018FEFA81AB80AC6010E94CA2DF4010F
:1013300081934F01882309F4CBC08C3741F4E2E05C
:10134000F0E0EC0FFD1FE00FF11F10820AC00F5FED
:101350001F4F65010730110519F7BAC0580101C0C8
:1013600056018201F8012081222309F4A8CF2130FF
:1013700009F04CC08181813049F46801F2E0CF0E60
:10138000D11CF80182810E94751E0AC0823051F47E
:101390006801F2E0CF0ED11CF80182810E94B61DD7
:1013A000860189C0833049F46801F2E0CF0ED11C78
:1013B000F80182810E94801DF3CF843019F00F5F05
:1013C0001F4F79C0F80122810E5F1F4F80E090E02F
:1013D00030E0205331092A30310568F4389EA001ED
:1013E000399E500D1124C901840F951F0F5F1F4FA7
:1013F000F8012081EDCF009709F45DC0EFE9FFE02F
:101400003197F1F700C000000197F5CFE22FF0E02F
:10141000E250FE4F2490822F86958695869590E027
:10142000FC01E251FE4F64902770712C022E02C025
:10143000759467940A94E2F7F1E06F227724FC0137
:10144000E252FE4F8490912C022E02C09594879414
:101450000A94E2F731E083229924FC01E253FE4F23
:10146000C490D12C02C0D594C7942A95E2F781E0AC
:10147000C822DD246114710419F081EE0E94B61DAA
:101480008114910419F086EE0E94B61D822D0E94EF
:10149000751E8114910419F086EE0E94801D61145E
:1014A000710419F081EE0E94801DC114D10419F05D
:1014B0008CE20E94751E0F5F1F4F54CF011537E756
:1014C000130709F042C181E00E942F1C0E94941E64
:1014D0008091D703877009F4F8C3F70182818823CC
:1014E00009F4F3C380911F0482FFEFC382E00E94DE
:1014F0003C1CEBC30115F7E71F0711F481E005C0A1
:10150000013027E7120721F482E00E94591CDECF48
:10151000F801E851FC47E730F10508F4E5C08823FD
:1015200009F470C110921104C8019057839708F014
:1015300013C184E090E00E94D22D90931F04809309
:101540001E04F801E150F047E232F10520F4EA5AB6
:10155000FF4F0C942C2E80911E048160ACC08091B2
:101560001F048860B4C080911E048260A4C0809172
:101570001E0420C080911E0488609DC080911F04BD
:101580001EC080911F048260A2C080911E048061F1
:1015900092C080911E0480628EC080911E0480647F
:1015A0008AC00E94681C80911E04806884C080915B
:1015B0001E04886084607FC080911F048260816007
:1015C00086C080911E048E7F76C080911F04877F25
:1015D0007EC080911E048D7F6EC080911E0420C04D
:1015E00080911E04877F67C080911F041EC0809178
:1015F0001F048D7F6CC080911E048F7E5CC0809123
:101600001E048F7D58C080911E048F7B54C00E94A1
:10161000681C80911E048F774EC080911E04877FC6
:101620008B7F49C080911F048D7F8E7F50C0809139
:101630001E0482FB222720F991E0922790FB82F979
:1016400090FB83F938C080911F04982F909591707A
:101650008E7F892B90FB81F93AC080911E0486FB16
:10166000222720F991E0922790FB86F924C00E945E
:10167000681C80911E0487FB222720F991E09227A5
:1016800090FB87F918C061E001C060E08EE090E057
:101690000E94D82D1EC080911E0484FB222720F9B1
:1016A00091E0922790FB84F906C080911E04982F48
:1016B000909590FB80F980931E040BC080911F04CD
:1016C00083FB222720F991E0922790FB83F98093F6
:1016D0001F0460911E0470911F0484E090E00E943A
:1016E000F62D0E94681CF4CEE858FF4F0C942C2E67
:1016F00006E221EE41EE6AE17CE723C007E225EE37
:1017000045EE6BE17CE71DC006E221EE40EE68E1AC
:101710007CE717C007E225EE44EE69E17CE711C0E3
:1017200006E221EE42EE6CE17CE70BC007E225EE1B
:1017300046EE6DE17CE705C008E221E045EE6EE192
:101740007CE7C7010E948C26C3CE013097E71907BA
:1017500009F0DECE82E0B8CE0631ECE71E0709F4D0
:1017600094C203309CE71907C9F1C0F40130FCE7CB
:101770001F07D1F100F501153CE7130709F047C039
:101780000E94681CFFEF24E33CE0F1502040304011
:10179000E1F700C000000E942B259ACE0B358CE7A4
:1017A000180761F10C359CE7190701F10A351C4750
:1017B00071F581E024C080911804982F9095917064
:1017C00090FB80F980931804992319F080E992E046
:1017D00002C08EE792E00E94A0077ACE6FEF7FEF03
:1017E00080E090E00E94F62D0E94420880911F0444
:1017F00082FB882780F991E0892701C080E00E9460
:101800002B1905C00631FCE71F0709F44EC2F7018A
:10181000828100811181882349F0C8010E94C91981
:10182000D82E682FC8010E94F71B04C0C8010E946F
:10183000C31BD82EB8018D2D0E9481160E948F16D1
:10184000B82E192F982EF7010281A580A2949FE04F
:10185000A9228091D7038770B9F00023A9F0812FC6
:10186000807F803421F080E28B0D883068F0809199
:101870001F0482FF09C082E00E943C1C8091D703B4
:101880008770DD24D3948111D12CC12EC2948FE0B6
:10189000C8228C2D90E08C30910508F0D8C1FC0155
:1018A000E158FF4F0C942C2E812F807F1F708823CE
:1018B00011F01295107F0023B9F0112309F4B5C17E
:1018C00080E28B0D883010F0911006C090914B0390
:1018D000192B10934B0305C090914A03192B1093B9
:1018E0004A030E949C18A1C18B2D0E94801D1123C8
:1018F00009F4ADC180E28B0D883088F1992079F12F
:10190000109590914A03192310934A032BC0812FFD
:10191000807F1F70803211F01295107F8B2D9920DF
:1019200029F0F1E09F1609F441C04FC080911F04D7
:1019300082FD1BC0002369F0112339F090914B0305
:10194000192B10934B030E949C1880E00E94B61D37
:101950007EC180E00E94801D112309F478C1812F8F
:101960000E9495180E949C1872C1002381F08091FA
:101970004C03AA2051F021E0A21207C0182B18171F
:1019800009F465C110934C0362C1812B16C0A110EC
:1019900003C00E948F1831C031E0A31609F457C16B
:1019A000812F0E94971C0E948F1851C1002341F083
:1019B00085E08A1508F44BC1812F0E949E1C47C107
:1019C00094E09A1508F443C118C0002349F0AA20F6
:1019D00099F3F701858180FF28C18F708583ECCF53
:1019E000AA2059F0893309F02FC1FFEF27EE33E029
:1019F000F15020403040E1F725C1812F0E94971C13
:101A000026C1812F86958695837019F0813061F00B
:101A10001EC1002321F08B2D912F937002C080E016
:101A200090E00E94562619C1002321F08B2D912FA2
:101A3000937002C080E090E00E9431260EC1602FBA
:101A40008B2D0E94A81C09C1812F8370A9F501115B
:101A500002C14B2D429546954770440F440F8B2D84
:101A60008F7090E09C01042E01C0220F0A94EAF7C7
:101A7000B4FE08C08FE090E001C0880F4A95EAF7F5
:101A8000809501C080E0169516951370123069F0AC
:101A900088F490914D03113019F0822B892302C0F4
:101AA000922B892B0E94651CD6C0822B90914D03EE
:101AB0008927F8CF822BF6CF002319F0812F817070
:101AC00001C08695882309F4C6C04B2D42954695E2
:101AD0004770440F440F8B2D8F7090E09C01042EB3
:101AE00001C0220F0A94EAF7B4FE08C08FE090E02C
:101AF00001C0880F4A95EAF7809501C080E01695ED
:101B000016951370123059F078F490910904113041
:101B100019F0822B892309C0922B892B06C0822BB6
:101B200090910904892701C0822B0E942C1C93C02C
:101B30001F70002339F0812F0E94591C8B2D0E94A9
:101B40009E1C89C08B2D0E94971C812F0E942F1CE8
:101B500082C08B2D92EF991681F1991538F0E0EF44
:101B60009E1659F0F1EF9F1619F15BC023EF921604
:101B700059F134EF9316C1F054C0002381F084E092
:101B80008A1508F464C01F7181E090E0012E01C045
:101B9000880F0A94EAF790910904892720C095E0FC
:101BA0009A1508F454C0EFCF80911F0482FD1AC02B
:101BB000002329F0812F8F7127C00023D9F3812FB3
:101BC0008F710E942F1C43C0002341F01F7181E0E0
:101BD000012E01C0880F0A94EAF701C080E00E943C
:101BE0002C1C35C0002399F01F71812F0E94591CB5
:101BF00080911F0482FF07C0E8E01E9FC0011124EE
:101C000083608093D703812F0E94591C20C081E0FC
:101C10000E943C1CF1E0FA15D0F482E00E943C1CCA
:101C200016C0002321F0AA2029F28B2D8FCEAA20E6
:101C300031F2893349F42FEF37EE83E02150304001
:101C40008040E1F700C000008B2D0E94801D88EFCE
:101C50008C0D843010F40E947B26DD20B1F1809140
:101C6000D70380FD32C0F701128285958595859551
:101C70000E94591CC7010E94F5088091D7038595E1
:101C8000859585950E942F1C20C080914B038A7AF0
:101C900091E009F490E09093C402811112C069E2CE
:101CA0008AE093E00E94EB2509C08091C402811173
:101CB0000AC069E28AE093E00E94B2250E949C1863
:101CC00007CC65E3EDCF65E3F5CF2D96E2E10C940B
:101CD000AF2D8295982F937344E0949F9001112427
:101CE0008C7C86958695282B822F8575880F2A7A7D
:101CF0002695822B0895AAE2B0E0E1E8FEE00C947C
:101D0000932D85B7806885BF85B7806885BF84B708
:101D1000877F84BF0FB6F894A89580916000886192
:101D200080936000109260000FBE90E080E80FB6D4
:101D3000F89480936100909361000FBE86EA93E26D
:101D40009093C3028093C2020E94CB210E94EA2199
:101D50008091E20084608093E20078948091FF0398
:101D60008823A1F01091E9001F709091EC00892F59
:101D7000817090FD80E8182B1092E9008091E800B6
:101D800083FD0E94B71E1F701093E90082E084BD9E
:101D900093E095BD9AEF97BD80936E001092C502B7
:101DA0001092C6021092C7021092C8020E949A2A8C
:101DB000811102C00E948A2A23982B988FE891E013
:101DC0000197F1F700C0000083B183FB882780F9F9
:101DD000809300010E944F1481110E942D2C80914C
:101DE000000180910001882311F090E001C095E08E
:101DF0009093DE0285E0891B8093DD0208E211E00A
:101E0000BDE2EB2EB1E0FB2ED8018D918D018F3F0D
:101E100011F00E94DB14E016F106B1F70DE211E0BB
:101E2000A6E3EA2EA1E0FA2EF80181918F018F3FFF
:101E300011F00E94DB14E016F106B1F784E1E6EF41
:101E4000F2E0DF01282F1D922A95E9F7E9ECF2E094
:101E5000DF011D928A95E9F780E090E00E94D22D83
:101E6000873E9E4F21F40E949A2A811102C00E944F
:101E70002D1882E090E00E94CA2D8093180484E01F
:101E800090E00E94D22D90931F0480931E040E9424
:101E9000F214EFE3FCE93197F1F700C000000E9473
:101EA000F2141B9B02C020E001C025E081E090E01D
:101EB00002C0880F991F2A95E2F72091F60230910F
:101EC000F70282239323892B41F06FEF7FEF80E0AD
:101ED00090E00E94F62D0E942B2583E090E00E9466
:101EE000CA2D0E94651C0E944F14811102C00E94DD
:101EF000302C81E091E09093150480931404F0E479
:101F00002F2E8091FF03853009F04AC081EA92E0CC
:101F10000E94A00700E112E18091FF03853009F0E3
:101F20003BC08091FF03843019F11092190428E11D
:101F300030E00FB6F894A895209360000FBE209271
:101F4000600083B7817F846083BF83B7816083BF74
:101F50007894889583B78E7F83BF0FB6F894A89541
:101F600080916000886180936000109260000FBED5
:101F70008091FE03882309F4CFCF0E94F214E6EF8C
:101F8000F2E081919191892B09F033C34AE053E04B
:101F90004E175F07B1F7C0CF0E94681C0E947B26D6
:101FA0000E94F214E1EEEE2EE2E0FE2E06EF12E0C9
:101FB00025EF32E0D801F701419151918D919D912A
:101FC000842795272E173F0719F0892BA9F322C0E4
:101FD000892B01F50E947D257C018091DF02909183
:101FE000E002E816F90609F4A5C08FEF89A38AA3D9
:101FF0001BA20E947D258160782F9DA38CA349A1FF
:102000005AA16BA18DA10E945808F092E002E092C3
:10201000DF0290C08091180481FD09C00E944F1416
:10202000382E76EF672E72E0772E512C44C085EB68
:1020300092E00E94A00756EFA52E52E0B52EC12CCB
:10204000D12C67EA862E62E0962EDF92CF9280EB4B
:1020500092E09F938F930E9439088DEA92E00E944C
:10206000A007F50180816180F2E0AF0EB11C0E94F3
:10207000690E782E862D0E94690E272D30E0322FB2
:102080002227A901482BCA019F938F939F928F9279
:102090000E94390885EA92E00E94A0075FEFC51A06
:1020A000D50A0FB6F894DEBF0FBECDBF9AE0C916B1
:1020B000D10459F6B3CFD3018D909D903D01F70126
:1020C000A080B180A824B924A114B10451F1412CFD
:1020D000CC24C394D12CC5018C219D21892BC1F026
:1020E0003320B1F04EA25FA221E0C4018C219D21DA
:1020F000892B09F420E028A70E947D258160782F94
:102100009AA789A74EA15FA168A58AA50E94580831
:102110004394CC0CDD1CF9E04F12DDCFD7018D923A
:102120009C925394B2E0EB0EF11CEAE05E12C3CF36
:102130000E9471250E944F1486E0E8E2F4E09E01BF
:102140002F5F3F4F7901D90101900D928A95E1F7F8
:1021500010922A0410922B0410922C0410922D0439
:102160008B81811104C08C81882309F45FC0809128
:102170002604909127040E946225AC0190912304CB
:10218000992339F02091260130E02417350758F0C3
:102190004DC0209127018AE0289F90011124241727
:1021A000350718F043C09F3F19F09F5F90932304B9
:1021B000DB80DD2061F00E94982B1D1414F491E067
:1021C00001C09FEF899F802D112480932A04DC8019
:1021D000DD2061F00E94982B1D1414F491E001C0E1
:1021E0009FEF899F802D112480932B0430912A0426
:1021F0003323E1F020912B042223C1F045EB34037B
:10220000C0011124992319F090932A0403C081E09E
:1022100080932A0455EB2503C0011124992319F05A
:1022200090932B0403C081E080932B048D81811156
:1022300004C08E81882309F453C0809124049091B6
:1022400025040E9462259C0190912104992309F4A0
:10225000EFC12135310508F443C09F3F19F09F5F5E
:1022600090932104DD80DD2061F00E945F2B1D141E
:1022700014F491E001C09FEF899F802D1124809379
:102280002C04DE80DD2061F00E945F2B1D1414F40D
:1022900091E001C09FEF899F802D112480932D0430
:1022A00030912C043323E1F020912D042223C1F03E
:1022B00045EB3403C0011124992319F090932C04A9
:1022C00003C081E080932C0455EB2503C001112449
:1022D000992319F090932D0403C081E080932D047D
:1022E00046E050E0B70188E294E00E944D2E892B31
:1022F000A9F480912A0481110FC080912B048111CF
:102300000BC080912C04811107C081E090912D04B5
:10231000911103C080E001C081E080FD0E94B32ADA
:1023200086E0F701A8E2B4E001900D928A95E1F70A
:102330000E947B26D82E8091F502D81631F1D092DA
:10234000F5020E9471258091180482FF1EC080FF53
:1023500004C083ED92E00E94A0078091180480FFE2
:102360000CC01F92DF928EEC92E09F938F930E949D
:1023700039080F900F900F900F908091180480FFF4
:1023800004C08CEC92E00E94A0078091FF0384308F
:1023900009F0B7CD83E08093E9008091E80082FFE7
:1023A000B0CD8091E80085FF21C00E94702381118B
:1023B0001BC080E2C82ED12C570109C08091F100CA
:1023C000D5018D935D01B1E0CB1AD10869F0809100
:1023D000E80085FDF3CF8091E8008B778093E800DB
:1023E0000E947023882399F391E001C090E08091CE
:1023F000E8008B778093E800992309F482CDE98186
:102400008E2F90E0FC013197E331F10508F0E8C030
:10241000E557FF4F0C942C2E1A828BE053C08A8113
:10242000823009F4FCC050F4813009F0D9C00E9418
:1024300071259B838C837D836E83D4C0833041F070
:10244000843009F0CDC01B821C821D821E82CAC04E
:10245000F701CE014596D8012C9111963C910E5F63
:102460001F4F3283238332968E179F07A1F7BAC07E
:102470008A81823021F0853009F4B4C0B1C06B810B
:102480007C818D819E810E94322E0E94662AAAC084
:102490004C816B818A810E9461279D83C7C02D81F9
:1024A0003E813227232732274C816B818A810E940B
:1024B000052798C00E942C2795C080E14EC081E07E
:1024C0008A838AE08B838EC00A811B8110270127B3
:1024D0001027AC80B12C6701C8018A509D4F96012E
:1024E0002E193F092A153B0508F07CC00A30B1E0DF
:1024F0001B0728F40E94CA2DF601848303C0D6016D
:1025000014961C920F5F1F4FBFEFCB1ADB0AE4CF6C
:102510000A811B81102701271027AC80B12C67018D
:10252000C8018A509D4F96012E193F092A153B0577
:1025300008F058C00A30E1E01E0728F4D6011496CE
:102540006C910E94D82D0F5F1F4FBFEFCB1ADB0A93
:10255000E7CF0E94F52646C084E08A8343C00A8103
:102560001B81102701271027AC80B12C6701C801FF
:10257000869696012E193F092A153B0598F5003DD0
:10258000E2E01E0730F40E94CA2DD60114968C9307
:1025900002C0F60114820F5F1F4FFFEFCF1ADF0A50
:1025A000E6CF0A811B81102701271027AC80B12CB0
:1025B0006701C801869696012E193F092A153B0529
:1025C00088F4003D22E0120728F4D60114966C919D
:1025D0000E94D82D0F5F1F4FBFEFCB1ADB0AE9CF48
:1025E0008FEF898340E250E0B70182E00E94BB2474
:1025F00088CC09BD19BD09B400FEFDCF8091D8007B
:102600008F7D8093D8008091E00082608093E0000D
:102610008091E00081FDFCCF0E94681C7DCC85E2AA
:1026200090E00E94CA2D1B821C821D828E83DACF0D
:102630002B30310508F013CE53CE90911E0492FF3B
:102640000DC0282F2871283019F4877F846006C0B8
:10265000282F2471243011F48B7F886093FF0DC0E4
:10266000282F2871283119F4877E846106C0282F0D
:102670002471243111F48B7E886120911F0420FF86
:102680000DC0382F3871383019F4877F816006C04B
:10269000382F3171313011F48E7F886021FF0DC0E9
:1026A000282F2871283119F4877E816106C0282FD0
:1026B0002171213111F48E7E886194FD877E089509
:1026C000EF92FF921F93CF93DF93CDB7DEB72B9797
:1026D0000FB6F894DEBF0FBECDBF7B0180E090E067
:1026E0000E94182D882309F463C040910C0150E02A
:1026F0004115510511F041E050E060910D017091DC
:102700000E0168597C4FCE010B960E945A2E4091C3
:1027100064035091650360916603709167032FB75E
:10272000F89480911A0490911B04A0911C04B0911C
:102730001D042FBF841B950BA60BB70B8436910588
:10274000A105B10538F489E693E00E94A01E9B859F
:10275000891781F181E090E00E94182D182F8823BD
:1027600091F04091140150E04B30510510F04AE0D7
:1027700050E0609115017091160168597C4FCE01AF
:1027800001960E945A2E89E693E00E94A01E91E0D5
:102790002B85281390E0192311F10E947125609375
:1027A00064037093650380936603909367030CC082
:1027B00010E001C011E08AE0E9E6F3E0DE011196E5
:1027C00001900D928A95E1F7112349F08AE0FE010C
:1027D0003196AAE5B3E001900D928A95E1F78AE07F
:1027E000EAE5F3E0D70101900D928A95E1F7812F98
:1027F0002B960FB6F894DEBF0FBECDBFDF91CF9101
:102800001F91FF90EF900895A0E0B0E0EAE0F4E1BE
:102810000C94992D7C015B01942E852E6901809189
:1028200059038A3018F001E010E002C00AE010E01D
:10283000C1E0D0E0B501C701F6010995811129C0B9
:1028400021960C171D078CF0CC9F9001CD9F300D69
:10285000300D112480E090E045E34A95F1F7000047
:10286000019628173907C1F7E5CF90911804892FF1
:10287000817090FF0FC08F929F9286E593E09F93A7
:102880008F930E9439080F900F900F900F9080E067
:1028900001C081E0CDB7DEB7ECE00C94B52D80919E
:1028A0005803811118C08091D80080618093D800AE
:1028B0008AE18A95F1F700C08091D90080FD02C0BD
:1028C00082E001C081E080935803823021F40E94AD
:1028D000CB211092FF0381E090915803913009F0D1
:1028E00080E00895A4E0B0E0E8E7F4E10C94A12DC5
:1028F00040917703509178036091790370917A0346
:102900002FB7F89480911A0490911B04A0911C0495
:10291000B0911D042FBF841B950BA60BB70B8436FB
:102920009105A105B10508F441C00E944F14882308
:1029300019F00E9471250EC00E9471250091C502F8
:102940001091C6022091C7023091C802600F711F1A
:10295000821F931FDC01CB010296A11DB11D89834B
:102960009A83AB83BC8380911A0190911B01885993
:102970009C4F4091190150E04530510510F044E062
:1029800050E0BE016F5F7F4F0E945A2E82E090E0C0
:102990000E94182D882359F00E94712560937703B7
:1029A000709378038093790390937A0381E024965F
:1029B000E4E00C94BD2DF894E82FE295EF70F0E080
:1029C00031A1282F2F7081E090E001C0880F2A9557
:1029D000EAF7982F9095932391A392A1892B82A334
:1029E00078940895AEE1B0E0E8EFF4E10C94952D11
:1029F000AE014F5F5F4F7A0184E1DA011D928A9543
:102A0000E9F708E211E06A016DE2462E61E0562E18
:102A100066246394712CE6E38E2EE1E09E2EF8018D
:102A200080818F3F09F446C0F894E82FE295EF705B
:102A3000F0E021A18F70A30102C0440F551F8A95B9
:102A4000E2F7CA01922F982B91A392A18095892336
:102A500082A3789400C0EDE2F1E021E030E0A12C07
:102A6000B12C41914F3F89F0A42FA295AF70B0E0F7
:102A700090968C9190E04F7002C0959587954A95FD
:102A8000E2F780FD02C0C90102C080E090E0A82A00
:102A9000B92A220F331F8E169F0619F7D8018C9181
:102AA0008F3F11F00E94DB14B0EABA95F1F7F601FE
:102AB000B182A0820F5F1F4FF2E0CF0ED11C4016F3
:102AC000510609F0ACCF44E150E0B70189EC92E047
:102AD0000E944D2E009741F024E1F701A9ECB2E0ED
:102AE00001900D922A95E1F70091DE02892B49F0C1
:102AF00081E0809350030E947D2590934F03809343
:102B00004E0380915003811102C0F12C24C08091AA
:102B10004E0390914F030E9462250597B0F310E099
:102B2000000F111F0A501D4F4AE050E069EC72E09F
:102B3000C8010E944D2E892B59F08AE0E9ECF2E0A1
:102B4000D80101900D928A95E1F7FF24F39401C01A
:102B5000F12C109250030E944F14E091DE02882362
:102B6000A9F16E0125E1C20ED11C8AE0D6011D92A9
:102B70008A95E9F70E2F10E0000F111F0A501D4F24
:102B8000E0905903B9E0BE1560F020E633E146E37A
:102B900051E0B601C8010E940414882309F47CC0E6
:102BA0000AC080915103909152030E946225843F94
:102BB000914058F78AC022E734E143E451E0B6017E
:102BC000C8010E940414811148C066C0F0E0EE0FF5
:102BD000FF1FEA50FD4F8AE0A9E6B3E001900D9295
:102BE0008A95E1F789E693E00E94A01E809368032E
:102BF0008090730390907403A0907503B090760357
:102C00008091530390915403A0915503B0915603C2
:102C100088169906AA06BB06D1F0809253039092BB
:102C20005403A0925503B09256030E944F14811191
:102C30000EC00E947125861A970AA80AB90A8092C6
:102C4000C5029092C602A092C702B092C80280E06C
:102C50008F296E96E0E10C94B12DB9E0BE1540F4D9
:102C60008091180480FF04C08DE093E00E94A007CB
:102C7000109259038091DD0290E0880F991F4AE07D
:102C800050E0B6018A509D4F0E944D2E21E02093C6
:102C90005703892B31F5DBCF809159038F3F19F012
:102CA0008F5F80935903809159038A3018F30E94F3
:102CB0007D2590935203809351038091180480FFE7
:102CC00004C080E293E00E94A0078091570388230C
:102CD00009F4BDCF8AE0D6011D928A95E9F71092DA
:102CE0005703A091DD02B0E0AA0FBB1FAA50BD4F51
:102CF0008AE0FE01759601900D928A95E1F781E0D8
:102D0000A7CF7A3048F4693038F4843028F4462F5D
:102D1000672F0E946127089580E090E00895CF9387
:102D2000DF938238910569F1B0F48133910509F49C
:102D300077C048F48932910509F469C08A32910557
:102D400009F473C092C08533910509F45BC08933DF
:102D50009105B9F08AC0833E910591F138F4803E27
:102D60009105D1F0823E910531F17FC0863E9105FB
:102D7000D9F1873E9105E9F1843E910509F075C0CE
:102D800028C020911E0420FD5BC021FD59C0209168
:102D90001F0423FD61C069C080911E0480FD4AC0EC
:102DA00080911F0480FF4CC080911E0484FD50C19F
:102DB00083EE90E04FC180911E0482FF3EC0F4CFAD
:102DC00080911E0482FD39C080911F0480FD38C0AF
:102DD000EBCF80911F0481FF39C080911E0484FDD8
:102DE00037C187EE90E036C180911E0483FF2BC06F
:102DF000F4CF80911E0483FD26C080911F0481FDC5
:102E000025C0EBCF80911E0485FD26C022C0809195
:102E10001E0485FD1EC080911F0483FF1DC00AC0D3
:102E200080911E0486FD1BC01DC080911E0486FD7E
:102E300019C015C089E390E00DC182EE90E00AC18F
:102E400080EE90E007C186EE90E004C184EE90E051
:102E500001C185E390E0FEC089E290E0FBC08AE218
:102E600090E0F8C081E390E0F5C0EC01811530E519
:102E7000930708F053C0811560E4960720F0CE0157
:102E80009F70906AE7C0803E910588F58D3C910562
:102E900018F0CE019065DEC0883A9105C0F4853AFD
:102EA000910550F08C2F855AC82FD0E0C25BDE4FC1
:102EB000888190E09064CEC08130910509F4C5C04E
:102EC00008F4C6C0049708F4C3C0CE01C3C0813C57
:102ED000910508F0BDC08C2F885AC82FD0E0CC0FC8
:102EE000DD1FCF5ADE4F888199819464B3C081156C
:102EF000904258F08D2F8F710E941D13282F2F7133
:102F0000CE0199279062922BA5C0C11581E0D80708
:102F1000E0F6C83ED10508F09BC0D7CFC03692E599
:102F2000D90708F053C0C03422E5D207B8F08C2F7F
:102F30008F718695869570E2879FA00111248C2F52
:102F4000837021E030E0B90102C0660F771F8A95D7
:102F5000E2F7CB019C68842B952B7CC0C03232E514
:102F6000D30740F08C2F8F7190E0982F8827816FC6
:102F7000906A70C0C11562E5D607B0F08C2F8695B7
:102F8000869520E2829FA00111248C2F837021E07E
:102F900030E0B90102C0660F771F8A95E2F7CB01D6
:102FA000842B952B9D6856C08C2F8F710E941D130A
:102FB00095E0D695C7959A95E1F7CF70D0E0DC2FD4
:102FC000CC27D0699E01282BC90144C0C03A72E5C4
:102FD000D70708F58C2F8F71C03892E5D907A8F470
:102FE0008695869570E2879F900111248C2F8370BF
:102FF00041E050E0BA0102C0660F771F8A95E2F700
:10300000CB019A68822B932B25C090E0982F8827BC
:10301000846F906A1FC0C03C22E5D20750F48C2F09
:103020008F710E941D138F7190E0982F88279062F6
:1030300011C0C03E32E5D30758F4CE018F719927F5
:10304000982F8827806F906A05C081E090E002C0C9
:1030500080E090E0DF91CF91089567EE7EEF80E011
:1030600090E00E94F62D60E082E090E00E94D82D72
:1030700060E083E090E00E94D82D10924D0360E064
:1030800074E184E090E00E94F62D60E086E090E03C
:103090000E94D82D6FEF87E090E00E94D82D40E08D
:1030A00050E0BA0188E090E00E94EA2D60E08DE0F7
:1030B00090E00E94D82D40E050E0BA0188E190E015
:1030C0000E94EA2D60E087E190E00E94D82D40E068
:1030D00050E0BA018CE190E00E94EA2D60E070E0DF
:1030E00080E290E00E94F62D40E050E0BA0188E1D5
:1030F00090E00E94EA2D80E00E946B2A0E948A2ABA
:1031000040E050E0BA018FE090E00E94EA2D40E0FC
:1031100050E0BA0183E190E00E94EA2D0895809189
:103120004C03811110924C030895809590914B03AC
:10313000892380934B030895EF92FF920F931F937F
:10314000CF9390914B0380914A03982B90930A035D
:1031500080914C038823D9F0892B80930A038091B6
:103160002101882331F080911E0487FF02C08EE187
:1031700001C086E0ECE0F3E090E0815028F021917E
:103180002223D9F39F5FF9CF91110E948F1840E25B
:1031900050E06AE273E08AE093E00E944D2E892BB2
:1031A00009F453C080E2EAE0F3E0AAE2B3E0019060
:1031B0000D928A95E1F7E0911404F091150430978F
:1031C00009F443C080912101882359F080911E04A5
:1031D00087FF07C080910A0380930B0386E08093EA
:1031E0000A030280F381E02D8AE093E00995809143
:1031F000180482FF2AC080FF04C08BEF92E00E9477
:10320000A0070AE013E0C8E085EFE82E82E0F82E80
:103210008091180480FF0CC0F80180811F928F9369
:10322000FF92EF920E9439080F900F900F900F902D
:10323000C1500F5F1F4FC111EBCF8091180480FF69
:1032400004C083EF92E00E94A007CF911F910F91DD
:10325000FF90EF900895CF9390911F0492FB222747
:1032600020F9281709F1C82F892FC0FB82F9809314
:103270001F0460911E0470911F0484E090E00E947E
:10328000F62D82E00E943C1C8091180480FF0CC047
:103290001F92CF938EED92E09F938F930E943908F7
:1032A0000F900F900F900F90CF9108958091D603BB
:1032B0009091A503891719F08F5F8770FBCF089550
:1032C0000F931F93CF93DF938091A40382958F7008
:1032D00009F05AC08091A103882309F455C0809158
:1032E000D6031091A50360919F037091A003C09134
:1032F000A203D091A30391E06F3F09F090E0292F42
:1033000006E0811709F440C0209721F07F3F21F0AB
:1033100030E003C031E001C0322F90E030FD31C019
:10332000089FF001099FF00D1124DF01AA55BC4F41
:1033300011963C911197371324C03C91361321C04C
:1033400012963C91129731111CC013964D915C91CD
:1033500014974C1B5D0B483C510598F48091A403D5
:103360008F7080618093A403E555FC4F80818F703E
:10337000806180838FE993E00E94F5080E945619CE
:1033800003C001968770BDCFDF91CF911F910F9140
:103390000895CF92DF92FF920F931F93CF93DF9305
:1033A0006C010091090480914D03082BC7E0D0E027
:1033B00010E0C8010C2E02C0959587950A94E2F79B
:1033C00080FD04C02197A8F7F12C09C0FC2EB6019E
:1033D0008C2F0E9481160E948F16019799F38F2DD2
:1033E000DF91CF911F910F91FF90DF90CF900895C3
:1033F000CF93DF93EC010E94C919BE010E94811690
:103400000E948F16DF91CF910895CF93FC018081A8
:10341000918123813481232B31F09F3F31F491E05E
:103420008F3F19F403C091E001C090E0C92FC17033
:1034300090FD1CC0808191810E94F81992959F7027
:10344000963079F010F4925001C09A50923088F47E
:10345000803F71F018F4883E60F40AC0843F49F45C
:1034600007C0883E28F0813F21F402C0C0E001C0BF
:10347000C1E08C2FCF910895A1E1B0E0E2E4FAE140
:103480000C949A2D8C0185E0F801DE011D960190C7
:103490000D928A95E1F7F801E28090919F03609187
:1034A000A0034091A2035091A3034115510531F0AF
:1034B0006F3F31F481E09F3F19F403C081E001C008
:1034C00080E0F82FF1709F2E80FD1BC1F801308144
:1034D0002181C380D4808FE9A82E83E0B82EF0909C
:1034E000A103F601E41BF50BFF2009F4C7C080918E
:1034F000A403E83CF10508F092C0482F407F09F092
:1035000051C0621311C093130FC0FE2CE1100CC008
:103510008F7080618093A403C5010E94F50880919B
:10352000A403F80185832AC1C114D10431F02F3FCF
:1035300031F481E03F3F19F403C081E001C080E035
:1035400080FD03C081E08E2502C080E090E0F82F6E
:10355000F170FF2E80FF1CC08091D6034091A5031F
:1035600056E0841709F4E8C090E0589FF001599F95
:10357000F00D1124EA55FC4F6181261306C06081CD
:10358000631303C06281E61203C001968770E9CF1E
:10359000FE2CEE2009F4F2C08091A4038160809398
:1035A000A40349C0621306C0931304C0E11002C013
:1035B000F80186C0C8010E94051A882351F1EE2047
:1035C00041F12091A403822F82958F7090E00297A1
:1035D00074F080919F039091A00398878F83198640
:1035E000DB86CA862C87CE0107960E94F50886E006
:1035F000F801AFE9B3E001900D928A95E1F70E94DE
:1036000060190AC06217C9F0C8010E94051A811129
:103610001EC0C8010E94F508FF24F394AFC0482FD4
:10362000407F81F78FE993E00E94F50886E0F5017D
:1036300011928A95E9F7F12CA1C09313E5CFE1101F
:10364000E3CFF8018583C8010E94F50854C0EE203D
:1036500001F32091A403822F82958F7090E002974E
:1036600034F280919F039091A0039A8389831B82F7
:10367000DD82CC822E83CE010196B7CFE83CF105E6
:10368000D0F5FE2CEE2029F2621327C0931325C03B
:103690002091A40320FD18C0822F82958F70482F9F
:1036A00050E04115510581F0F80125834F30510557
:1036B00041F08F5F982F9295907F822F8F70892B8A
:1036C0008583C8010E94F50886E0F801AFE9B3E000
:1036D00001900D928A95E1F751C0C8010E94051A28
:1036E000811185CF8091A40381608093A403C801D8
:1036F0000E94F50843C086E0F50111928A95E9F72A
:103700003DC0EE2009F485CFC8010E94051AF82EAD
:10371000882309F47ECF86E0F801AFE9B3E0019099
:103720000D928A95E1F780919F039091A0030E94EA
:10373000F8190E94601922C03D872E878D859E85CD
:103740000E94F819292F22952F70223028F49F709B
:1037500039F0811105C00BC0243028F49F7049F462
:10376000805E883020F0C8010E94F5089F2CF92C5B
:1037700005C0F8019581907F99F7F9CF8F2D61965B
:10378000EBE00C94B62D292F9A3078F5893068F546
:1037900090E039E0239F800D911D1124682F677000
:1037A00023E0969587952A95E1F7FC01EE0FFF1F20
:1037B000E80FF91FE558FC4F40E050E080E0219110
:1037C00030E0062E02C0369527950A94E2F7217064
:1037D0003327042E01C0220F0A94EAF7822B4F5F91
:1037E0005F4F4330510559F7089580E00895292F20
:1037F0009A3088F5893078F590E039E0239F800D84
:10380000911D1124282F277051E001C0550F2A95D2
:10381000EAF723E0969587952A95E1F7FC01EE0FEC
:10382000FF1FE80FF91FE558FC4F20E030E070E083
:103830004081CB01022E02C0969587950A94E2F74B
:103840008170819584278523842781932F5F3F4F43
:103850002330310569F7089580930904089521E024
:1038600030E001C0220F8A95EAF720958091090483
:1038700082230E942C1C08952091D70380958223D7
:103880008093D703982F977099F430E0482F082E33
:10389000000C550B2417350759F090911F0492FF27
:1038A00007C08595859585950E942F1C1092D7039A
:1038B000089521E030E001C0220F8A95EAF7809157
:1038C0000904822B0E942C1C089580934D030895B7
:1038D00010924B0380912101882331F080911E04C6
:1038E00087FF02C08EE101C086E0ECE0F3E0DF017B
:1038F0001D928A95E9F780E090E00E94562680E0CC
:1039000090E00E94312610924A030E949C18E8E23F
:10391000F4E086E0DF011D928A95E9F71092230416
:1039200010922104109222040E94B32A0895882341
:1039300021F00E9495180E949C180895882339F060
:1039400090914B03892B80934B030E949C18089500
:10395000662309F45CC08D3C21F40E94982B81956C
:1039600004C08E3C29F40E94982B80932B04C5C080
:103970008F3C21F40E94982B819504C0803D29F44E
:103980000E94982B80932A04B8C0893D19F40E94A4
:103990005F2B05C08A3D31F40E945F2B8195809397
:1039A0002C04ABC08B3D21F40E945F2B819504C099
:1039B0008C3D29F40E945F2B80932D049EC09FE2D2
:1039C000980F983078F421E030E0A90102C0440F4C
:1039D000551F9A95E2F7CA0190912904892B80938B
:1039E00029048BC08D3D21F48091220481600CC09C
:1039F0008E3D21F480912204826006C08F3D09F043
:103A00007CC08091220484608093220476C08D3C27
:103A100039F490912B0497FF35C010922B0459C0B4
:103A20008E3C29F490912B041916BCF32BC0909175
:103A30002A048F3C29F497FF25C010922A0449C01C
:103A4000803D19F41916CCF31DC090912C04893DCA
:103A500029F41916BCF410922C043BC08A3D19F4C9
:103A600097FF10C0F8CF8B3D39F490912D0497FF4C
:103A700009C010922D042DC08C3D21F490912D048D
:103A80001916BCF39FE2980F983080F421E030E0E3
:103A9000A90102C0440F551F9A95E2F7CA0180950B
:103AA0009091290489238093290413C08D3D21F42A
:103AB000809122048E7F0BC08E3D21F480912204E0
:103AC0008D7F05C08F3D29F4809122048B7F8093E8
:103AD000220480912A04811106C080912B04811157
:103AE00002C01092230480912C04811106C08091A1
:103AF0002D04811102C0109221040E94B32A08955E
:103B0000882399F19CEF980F913A30F4682F8AE05E
:103B100093E00E94B2250DC090E2980F983060F4B7
:103B2000877091E001C0990F8A95EAF7892F0E946A
:103B300095180E949C1808959BE5980F933028F4DF
:103B400080E090E00E945626089598E5980F9931FC
:103B500028F480E090E00E943126089593E3980FC6
:103B6000933118F460E00E94A81C0895CF93882335
:103B700009F4B9C0C82F8CEF8C0F813AF0F5809111
:103B80002E04813081F030F08230A1F58C2F0E941C
:103B9000A827A9C080914B03823209F06CC08C2FFA
:103BA0000E94EC2866C080914B038232C1F3C4317D
:103BB000C9F058F4CB3069F0C031B9F482E0809399
:103BC0002E0488E30E94A82752C0C93259F0C83396
:103BD00061F48BE09DE00E94A0078EE693E00E94D6
:103BE000A00745C010922E043FC08CE693E00E94CF
:103BF000A0073AC010922E043EC080E28C0F88309D
:103C000078F4C77081E090E001C0880FCA95EAF7A8
:103C100090914B03892B80934B030E949C1863C0A7
:103C2000EBE5EC0FE33040F4F0E0E25BFE4F808127
:103C300090E00E94562657C0E8E5EC0FE93150F4B9
:103C4000F0E0EE0FFF1FEF5AFE4F808191810E943E
:103C5000312649C083E38C0F833108F044C061E012
:103C60008C2F0E94A81C3FC080E0817002C081E0C0
:103C7000FCCF811138C0809121018823E1F080912F
:103C80001E0487FF18C0EC2FE695E695E695F0E058
:103C9000E65FFC4F8281282F30E04C2F477081E097
:103CA00090E002C0880F991F4A95E2F78223932380
:103CB000892B61F412C0ECE0F3E082E193E0219102
:103CC000C21721F08E179F07D1F707C06C2F8AE02B
:103CD00093E00E94B2250E949C186C2F8AE093E02A
:103CE0000E94EB259ACFCF9108951F93CF93DF9336
:103CF000182F893319F0C0E0D0E002C0C0E5D0E051
:103D0000812F0E94B61D209741F08FE99FE0019717
:103D1000F1F700C000002197F6CF812F0E94801D8F
:103D2000DF91CF911F91089580910904982F96708B
:103D3000963011F4886001C0877F0E942C1C089582
:103D4000FC01AC01465F5F4F8FEF91E32191822729
:103D500028E030E087FF03C0880F892701C0880F63
:103D600021503109B9F7E417F50781F70895AAE260
:103D7000B0E0EDEBFEE10C94A22DE1E0F4E08091E7
:103D8000F100819344E0E930F407C9F7809102041F
:103D9000833009F463C030F4813071F0823009F46B
:103DA0009DC0B4C08A3009F489C08B3009F46EC05C
:103DB000893009F0ABC020C080910104813A09F03C
:103DC000A5C08091E800877F8093E800809105047A
:103DD00090910604892B21F460E28DED93E003C0FD
:103DE00060E080E090E070E00E945D248091E80057
:103DF0008B778093E8008AC080910104813209F0BA
:103E000085C08091050490910604009719F00297EF
:103E100009F07CC08091E800877F8093E800809162
:103E2000E80082FD05C08091FF038111F8CF6EC0CC
:103E30002091F3008091F20090E0922B029731F4F0
:103E40008091F100813011F0863021F48091F100F1
:103E50008093DC038091E8008B7754C0809101044B
:103E6000813A09F053C08091050490910604892B92
:103E700009F04CC08091E800877F8093E800809132
